:100000003DC04AC049C048C047C046C045C044C0C2
:1000100043C042C0010A2A4B7A85FF01020305074B
:10002000FBFAFE01020305070000000705030201B9
:10003000000000020407FBFAFEF6000204070000BD
:10004000000000070402000000000001020306FB9C
:10005000FAFEF6010203060000000006030201009A
:1000600000000002030507000000000704FB000079
:1000700000000007007993A3ADB8FF0011241FBE54
:10008000CFE9CDBF10E0A0E6B0E001C01D92AE36D2
:10009000B107E1F7C2D0B2C1B3CF815019F492E0F9
:1000A00093BF02C0813011F491EA9FBDE82FF0E0C8
:1000B000EC5EFF4FE491E9BD089526EB33E003C009
:1000C000F9013197F1F70197D8F7089588EE93E099
:1000D000F4CF369A3699FECF85B10895CF93C0916B
:1000E00068008C2F8F5F8F7180936800609169002A
:1000F00090E076D16FEF8C2F90E0CF9171C1EEDF61
:1001000060916C008FE390E06BD160916B008EE3A7
:1001100090E066D160916A008DE390E061C1CF9379
:10012000109268001DC08C2F90E052D18F3FA9F033
:10013000809369008FE390E04BD1C82F80936C00CF
:100140008EE390E045D180936B008DE390E040D149
:1001500080936A00CC3070F007C0CF5FC093680016
:10016000C0916800CA33F8F21092690010926C00D6
:10017000CF91C5CFCF910895E0916C00F0E083E07E
:10018000EE0FFF1F8A95E1F7E55EFF4F80E0A0E6E6
:10019000B0E003C09D933196822F883008F005C0EF
:1001A0009491282F2F5F9111F5CF80936D000895C2
:1001B000811102C019BC089570CF08951F93CF9389
:1001C000DF93182FEB010AC083E067DFCE0175DFF4
:1001D00019BCCE0172DFCE0170DF11501111F4CFC6
:1001E000DF91CF911F9108951F93CF93DF93EC017F
:1001F000862F6BEB70E0E2DF888111E08127888336
:100200007EDF6FE070E080E2D9DF8881812788831C
:1002100076DFDF91CF911F9159CFB99A83EA8FBDD5
:1002200081E083BF7CDFA8DF80916A0081111AC062
:1002300080916E00803270F48F5F8F7180936E00BA
:10024000809169008F5F8093690090916D0089179C
:1002500048F006C010926E0080916B00811102C0C0
:10026000109269003BDFA29A81E687B986EC86B9D5
:10027000369AC0916900EC2FF0E0E05AFF4FD08130
:1002800080916A00882319F010926E0001C0CD2F72
:1002900010E09DEFF92E80916E008A30B8F016DFE5
:1002A00010926E00F092690061E08AE690E09CDFB7
:1002B0001092690062E08BE690E096DFE0916900C1
:1002C000F0E0E05AFF4FC081DC2F5DC0CB3F69F406
:1002D00008E087E0E2DE81E290E0EFDE19BC83E433
:1002E00090E0EBDE0150A9F74EC0CA3F71F404E084
:1002F00087E0D3DE8AE090E0E0DE84E0CEDE8CE3CF
:1003000090E0DBDE0150A1F712C0C63F91F468EC2B
:1003100070E083E053DF88EE93E0CFDE64EF71E0BE
:1003200083E04CDF68EC70E083E048DFCFDECEDEB8
:100330002AC0CE3F79F4CDDE982F80E001C08F5FD8
:10034000E82FF0E0EB58FF4FE491E917C0F36BEBB7
:1003500070E0EBCFCD3F91F41092690010926A00EB
:1003600000E000936C00CBDE0F5F6BEB70E0802F42
:1003700025DFACDEABDE0C30A1F7D9CF8D2F18DF37
:1003800084EF91E09ADE10926E00349B84CF85B1A9
:100390008937D8F41F5F1830C8F0D83088F4D230CD
:1003A00010F0D1500EC019BC85B7877E806185BF23
:1003B00085B7806285BF889585B78F7D85BF01C071
:1003C000D3E08D2FF5DE82DECD2F10E0369A63CF9D
:1003D000E199FECF1FBA8EBBE09A99278DB308959D
:1003E000262FE199FECF1CBA1FBA8EBB2DBB0FB6CC
:1003F000F894E29AE19A0FBE01960895F894FFCF1F
